:020000040000FA
:10000000830100308A001928A00003088301D7006B
:100010000A08D8008A010B1D11288A11A9268A1105
:100020000B11831258088A0057088300A00E200E77
:100030000900A1308400A1302F20213084005530E8
:100040002F200730DA00FF30D900553084005630B9
:10005000332083018A11F52E04068001840A0406E8
:10006000031D2C280034D6008A113F208A118000FD
:10007000840A04085606031D34280034D900DA1B0C
:1000800048285A088A005908D90A0319DA0A82004E
:1000900083135A1883175908D90A840000080800E6
:1000A00082075234653476342E342034563430345A
:1000B0002E3432342034203443346F347034793465
:1000C00072346934673468347434203432343034F0
:1000D000303431342D34323430343034333420340D
:1000E0004E3469346E34743465346E3464346F3431
:1000F00020346F346634203441346D3465347234C6
:100100006934633461340034FF3FFF3FFF3FFF3FFA
:10011000FF3FFF3FFF3FFF3FFF3FFF3FFF3FFF3FEF
:10012000FF3FFF3FFF3FFF3FFF3FFF3FFF3FFF3FDF
:10013000FF3FFF3FFF3FFF3FFF3FFF3FFF3FFF3FCF
:10014000FF3FFF3FFF3FFF3FFF3FFF3FFF3FFF3FBF
:100C600083122308031D472E07108711D401D40ACD
:100C700014305402031C372E8715D401D40A3230A5
:100C80005402031C3E2E071A472E03100800D401FD
:100C90002108540203188B2E5408333E84000008A8
:100CA000D300531C552E8714562E87100714071097
:100CB000D31C5C2E87145D2E871007140710531D5C
:100CC000632E8714642E871007140710D31D6A2E15
:100CD00087146B2E871007140710531E712E87146C
:100CE000722E871007140710D31E782E8714792EC2
:100CF000871007140710531F7F2E8714802E87102C
:100D000007140710D31F862E8714872E8710071409
:100D10000710D40A482E2308023A031D9B2ED40143
:100D200007140710D40A0A305402031C902E071926
:100D30009F2E03100800071A9F2E031008000314AB
:100D400008008312051224088600851585110516F2
:100D50000800831298130930831699009813181706
:100D60009812181683121817181218169812D5010F
:100D7000071BB82E071BB82E071BB82E071BB82E53
:100D80008C129817080020308312850083160514F2
:100D90008514051185110512851283128516FF3001
:100DA000860083168601DF308312870083160710C2
:100DB00087100715871107168712071787178312E1
:100DC00005080339A40083168112811101158110D1
:100DD00001148B1683128101A92683160C128C1222
:100DE00083128C120B178B170800C3268A11E92F68
:100DF0008C1EE92F181C042F81011A082406031DDC
:100E0000E92FD501D50A072F1A08A900E92F8C1E52
:100E1000E92F181C382FCB2FD500E92F0511A80179
:100E20000230D500912F05150F2FA3011C2FA30110
:100E3000A30A1C2F0230A3000330D500942F87167D
:100E4000292F8712292F8512292F8516292FA401D2
:100E5000A1262408A6005B100330A70005300C2F44
:100E6000A401A40A282F0230362F0330A400282F13
:100E70001A08A500D600103056020318E92F0730D3
:100E80008A004630560703188A0A8200292F0E2F3F
:100E9000132F152F172F1A2F1F2F212FE92FE92F6F
:100EA000232F252F272F302F332F352F1818902F32
:100EB000A819622F28082B3E84001A088000A50775
:100EC000A80A912F1A082506031D8D2F2B088600CE
:100ED000851585112C088600851585112D0886003D
:100EE000851585112E088600851585112F08860029
:100EF0008515851130088600851585113108860015
:100F00008515851132088600851585112408A600EF
:100F10005B100330A7000530112F24088038872F7D
:100F2000A9268C1EE92F562F8C1EE92F1818CB2FBF
:100F30001A08A100A50721302102031CA22F81015C
:100F40008B16E82FA2010430D5008C1EE92F18184B
:100F5000CB2F203022020318B52F2208333E840005
:100F60001A088000A507A20AE92F1A082506031D02
:100F7000E82F30262408031CC92FA6005B1003307D
:100F8000A7000530D5002308023A031DE92FA1264A
:100F9000E92F80382A2FA926E92FA70BE92F18124D
:100FA00083169817981683125B1CD92F8316181472
:100FB000DB2F8316181083122608990006300C2F99
:100FC0008316981CE92F9812981383128C12181606
:100FD000D501640083125508D60007305602031865
:100FE000E92F07308A00F830560703188A0A820072
:100FF000F82E072F912F942FA52FCD2FE02F0034FF
:10100000FF3FFF3FFF3FFF3FFF3FFF3FFF3FFF3FF0
:10101000FF3FFF3FFF3FFF3FFF3FFF3FFF3FFF3FE0
:10102000FF3FFF3FFF3FFF3FFF3FFF3FFF3FFF3FD0
:10103000FF3FFF3FFF3FFF3FFF3FFF3FFF3FFF3FC0
:00000001FF
